:100000004AC086C063C062C061C060C05FC05EC0DD
:100010005DC05CC05BC05AC059C058C057C056C014
:1000200055C054C053C000CDD914F13C28E5A16C93
:1000300078B5509D89441A03540069006C006C0027
:1000400020004800610072006200610075006D00D0
:100050001A036900320063002D00740069006E000D
:1000600079002D0075007300620012011001FF007D
:100070000008030431C60502010200010902120052
:1000800001010080050904000000FF0000000403D6
:1000900009040100FF8E11241FBECFE5D4E0DEBFAE
:1000A000CDBF10E0A0E6B0E0ECE2F9E002C00590C0
:1000B0000D92A636B107D9F710E0A6E6B0E001C070
:1000C0001D92A639B107E1F7EDD22EC499CFDC011C
:1000D0009FEF8FEF660FB9F046E2F0E0229560FFE8
:1000E0002D91E82FE227EF70929582958F70392F2E
:1000F000307F832B9F70E40F3591932731709327C6
:1001000083276A9559F7809590958D939D930895CF
:100110000F931F932F93DF93CF930FB70F93829972
:10012000FECF82990BC0829909C0829907C082993B
:1001300005C0829903C000E40ABFA8C0C0917E0038
:10014000DD27C158DF4F0BE014E124E0829BE9CFAB
:100150003F934F936F9360B330E803C060B3432B7A
:100160004993442764712627215020B32471A9F1B3
:1001700037953C3FA0F56227615060B364713795B5
:100180003C3F98F526272150379520B324713C3FFA
:1001900090F56227615037953C3F60B36471A0F5DC
:1001A0002627215037953C3FC8F520B3247162279C
:1001B000615037953C3FB0F50A9560B37AF06471B1
:1001C0002627215037953C3F88F520B324716227BC
:1001D000615037953C3F10F22DC031C048C06127B7
:1001E00020B324713F774160C6CF3F77426060B350
:1001F00064712127C7CF3F774460612720B3247102
:10020000622761503795C8CF3F774860212731601A
:1002100060B36471262721503795C6CF3F77406180
:100220006127C1CF3F7740622127C4CF3F77406429
:100230006127C9CF3F774068212700C08FCF30E4C6
:100240003ABF0B500195033090F0C01B2881233C2E
:1002500091F12B3481F119811F774091950014178A
:1002600031F42936D9F02D3249F0213E39F04427B6
:10027000409366006F914F913F9108C020936600B4
:100280006F914F913F910AB706FD49CF0F910FBF74
:10029000CF91DF912F911F910F91189500917000D0
:1002A0000023F1F040917D004423D1F4409370008D
:1002B000C1E7D0E018C0209166002223C1F240912E
:1002C0007D00442369F400937D0020937C0000911D
:1002D0007E004BE0401B40937E00C0E6D0E002C0B1
:1002E000C1E6D0E001E022B32B7E206111B314619E
:1002F00022BB11BB14E130E830FF212722BB379528
:1003000047954C3FC0F530FF2127379522BB4795D5
:100310004C3FA8F530FF21273795000022BB4795B9
:100320004C3F78F530FF21273795000022BB4795D9
:100330004C3F48F530FF2127699122BB37954795FF
:100340004C3F18F530FF2127379522BB47954C3F8E
:1003500000F530FF21273795479522BB4C3FD8F455
:1003600030FF21273795362F479522BB4C3FA8F405
:100370000A9512F614C02127442722BBC2CF212799
:10038000C5CF2127CBCF2127D1CF2127442722BB7F
:10039000D7CF2127DACF2127DFCF2127E5CF2B7E2B
:1003A00022BB6F914F913F9100E40ABFDF91CF9143
:1003B00011B3022F206122BB1B7EDFBFDF912F9183
:1003C000000011BB02BB1F910F91189585B7836088
:1003D00085BF8BB780648BBF789408951F93CF93AC
:1003E000DF9360917D00662309F477C080917E00E1
:1003F000CCE0D0E0C81BD109C158DF4F81E0809329
:10040000670080917C008D3209F059C01E818F8178
:1004100081111FEF8881807609F041C0898188238E
:1004200021F41882198292E042C0853021F48A8139
:1004300080936B00BAC0863039F582E08093670004
:100440008B81813021F492E1CAE6D0E030C0823065
:1004500021F492E1CCE7D0E02AC0833009F0A5C0B6
:100460008A81882321F494E0CEE8D0E020C0813056
:1004700021F49AE1C6E3D0E01AC0823009F095C0B9
:100480009AE1C0E5D0E013C0883019F481E0888398
:1004900004C08A3009F089C0188291E008C0CE01FA
:1004A000ADD1982F8F3F19F483E08093670019171F
:1004B00008F0192FD0936A00C093690005C06350FB
:1004C00011F0CE0112D110E01093680083EC8093FC
:1004D00071001092700010927D008091700088234E
:1004E00009F053C020916700222309F44AC080918B
:1004F000710098E889278093710010916800193085
:1005000010F018E002C0112379F1233031F482E7B2
:1005100090E0612F28D1182F22C0309169004091BE
:100520006A00213061F4832F942FFC01A2E7B0E030
:1005300081918D938E2F831B8117D0F30CC0832F55
:10054000942FFC01A2E7B0E0849131968D938E2F19
:10055000831B8117C8F3F0936A00E09369008091D0
:100560006800811B8093680082E790E0612FAFDD17
:100570001D5F109370001350183038F4109267000C
:1005800004C080916B00809395008AE002C0815086
:1005900019F0849BFCCF0BC0F8941092700010925D
:1005A0007D0010926B00789402C090E082CFDF91C2
:1005B000CF911F910895882319F0A498AC9A0895BB
:1005C000A49AAC980895E0916400F0916500319789
:1005D000F1F7882329F0A598AD9A9D9BFECF02C024
:1005E000A59AAD9880916200909163000197F1F710
:1005F000089581E0E8DF80E0E6DF089580E0DBDF5A
:1006000081E0E1DF81E0D7DF08950F931F93CF935F
:10061000DF93C7E0D0E0082F10E0C8010C2E02C025
:10062000959587950A94E2F780FF02C081E001C0AA
:1006300080E0C1DFDEDF21978FEFCF3FD80769F77A
:1006400081E0B9DF81E0BFDF13B380E0BCDF12954A
:100650001F701095812F8170DF91CF911F910F91A5
:100660000895FF920F931F93F82E81E0A4DF80E09E
:10067000AADF17E000E081E0A6DF000F9C9901608F
:1006800080E0A1DF1150B8F7FF2011F081E001C038
:1006900080E091DFAEDF81E08EDF802F1F910F9130
:1006A000FF9008952EE088E190E00FB6F894A895A9
:1006B00081BD0FBE21BDA498AC9AA598AD9A1092A9
:1006C0006E0010926D0082B38B7E82BB81B3846119
:1006D00081BB80E49CE90197F1F781B38B7E81BBFC
:1006E00075DE7894A8957ADEFDCFEF92FF920F9396
:1006F0001F93CF93DF93E82E292FF62E80916C0065
:10070000813021F500916D0010916E00862F90E0F0
:100710000817190708F4F02E8E2D922F9C01E9017D
:1007200002C0899172DF9E012E192F15D0F3A80106
:100730004F19510950936E0040936D0080916F00E6
:1007400081FF0AC0452B41F459DF06C08E2D60E0C1
:1007500070E04F2D50E0E1D0DF91CF911F910F91CC
:10076000FF90EF900895CF92DF92EF92FF920F9358
:100770001F93CF93DF93C82E292FD62E80916C0024
:10078000813061F5E0906D00F0906E00862F90E072
:10079000E816F90608F4DE2C8C2D922F9C018901B5
:1007A000E70108C080E0209709F481E05ADFF801F2
:1007B00081938F012197802F8C198D1598F39701C4
:1007C0002D19310930936E0020936D0080916F00D8
:1007D00081FF0AC0232B41F411DF06C08C2D60E09D
:1007E00070E04D2D50E099D08D2DDF91CF911F916C
:1007F0000F91FF90EF90DF90CF9008951F93CF93CC
:10080000DF93EC0189818230E9F0833030F4882372
:1008100059F0813009F073C00DC0833009F46AC00B
:10082000883008F06CC030C08A8188838B818983CE
:1008300082E066C0CE0162E970E044E050E064D03E
:1008400084E05EC08A819B81909363008093620004
:10085000892B31F481E090E09093630080936200F3
:1008600080916200909163009695879590936500C2
:1008700080936400892B09F042C081E090E090935E
:100880006500809364003BC01C81110F8A8180FD4C
:100890001160898180FD04C081E08DDE81E093DEFE
:1008A00080E089DE80E08FDE812FAFDE882341F497
:1008B00082E080936C0010926E0010926D0010C068
:1008C00081E080936C002E813F8130936E002093F5
:1008D0006D00898180936F0081FF03C0232B09F491
:1008E0008DDE8A8180FF0BC08E819F81892B39F03C
:1008F0008FEF06C080916C00888381E001C080E0AA
:10090000DF91CF911F910895FB01DC0102C005909A
:100910000D9241505040D8F70895DC0101C06D930D
:0C09200041505040E0F70895F894FFCFDC
:06092C00D25A0A0005008A
:00000001FF
